:020000040000FA
:0408000036EF08F0D7
:1008100003B213EF05F0F2B42EEF05F09EB036EF01
:1008200005F09EB23EEF05F0F2A81AEF04F0F2B226
:1008300025EF04F0F2A620EF04F0F2B022EF04F06E
:10084000E5EF07F0F296F290FF00CD90F2929EA0B5
:100850002FEF04F00101533F2FEF04F0542BAEC1F2
:10086000B2F1AFC1B3F1B0C1B4F1B1C1B5F1AAC138
:10087000AEF1ABC1AFF1ACC1B0F1ADC1B1F1A6C148
:10088000AAF1A7C1ABF1A8C1ACF1A9C1ADF1A2C158
:10089000A6F1A3C1A7F1A4C1A8F1A5C1A9F19EC168
:1008A000A2F19FC1A3F1A0C1A4F1A1C1A5F19AC178
:1008B0009EF19BC19FF19CC1A0F19DC1A1F196C188
:1008C0009AF197C19BF198C19CF199C19DF1CECF4E
:1008D00096F1CFCF97F153C198F154C199F1CF6AF6
:1008E000CE6A0101536B546B9E90CD800FBC0F8E6E
:1008F0000FBA7EEF04F00F8AE5EF07F00F8C0FBE02
:10090000BAEF04F096C19AF197C19BF198C19CF19E
:1009100099C19DF19AC19EF19BC19FF19CC1A0F12B
:100920009DC1A1F19EC1A2F19FC1A3F1A0C1A4F1FB
:10093000A1C1A5F1A2C1A6F1A3C1A7F1A4C1A8F1CB
:10094000A5C1A9F1A6C1AAF1A7C1ABF1A8C1ACF19B
:10095000A9C1ADF1AAC1AEF1ABC1AFF1ACC1B0F16B
:10096000ADC1B1F1AEC1B2F1AFC1B3F1B0C1B4F13B
:10097000B1C1B5F101015E6B5F6B606B616B96514C
:100980005E2797515F2398516023995161239A51B3
:100990005E279B515F239C5160239D5161239E5193
:1009A0005E279F515F23A0516023A1516123A25173
:1009B0005E27A3515F23A4516023A5516123A65153
:1009C0005E27A7515F23A8516023A9516123AA5133
:1009D0005E27AB515F23AC516023AD516123AE5113
:1009E0005E27AF515F23B0516023B1516123B251F3
:1009F0005E27B3515F23B4516023B5516123D89072
:100A00000101613360335F335E33D890010161339C
:100A100060335F335E33D8900101613360335F33FD
:100A20005E33E5EF07F00392030103EE00F080511F
:100A30007F0BE92604C0EFFF802B8151805D700B96
:100A4000D8A48B8200008051815D700BD8A48B925A
:100A500081518019D8B40790E5EF07F0F2940101B5
:100A6000453FE5EF07F0462BE5EF07F09E900101CB
:100A7000533FE5EF07F0542BE5EF07F09E9204009B
:100A800062A143EF05F007B492EF05F01EC620F611
:100A90001FC621F61CC61EF61DC61FF61AC61CF67A
:100AA0001BC61DF606C608F607C609F604C606F6F6
:100AB00005C607F602C604F603C605F626C628F6DE
:100AC00027C629F624C626F625C627F622C624F60A
:100AD00023C625F60EC610F60FC611F60CC60EF686
:100AE0000DC60FF60AC60CF60BC60DF62EC630F66E
:100AF0002FC631F62CC62EF62DC62FF62AC62CF69A
:100B00002BC62DF616C618F617C619F614C616F615
:100B100015C617F612C614F613C615F6B6EC27F06E
:100B20004EEC27F0077C07ACADEF05F0C274C2B401
:100B3000A7EF05F0C3CFB3F5C4CFB4F50501D89046
:100B4000B433B333D890B433B333AEEF05F0C3CF7F
:100B500055F1C4CF56F1AEEF05F0C28207B41BEFDA
:100B600006F047C14BF148C14CF149C14DF14AC1B2
:100B70004EF15EC162F15FC163F160C164F161C1B8
:100B800065F196C1B6F197C1B7F198C1B8F199C1B5
:100B9000B9F19AC1BAF19BC1BBF19CC1BCF19DC135
:100BA000BDF19EC1BEF19FC1BFF1A0C1C0F1A1C105
:100BB000C1F1A2C1C2F1A3C1C3F1A4C1C4F1A5C1D5
:100BC000C5F1A6C1C6F1A7C1C7F1A8C1C8F1A9C1A5
:100BD000C9F1AAC1CAF1ABC1CBF1ACC1CCF1ADC175
:100BE000CDF1AEC1CEF1AFC1CFF1B0C1D0F1B1C145
:100BF000D1F1B2C1D2F1B3C1D3F1B4C1D4F1B5C115
:100C0000D5F1B3C5B5F5B4C5B6F5B5C5B7F5B6C537
:100C1000B8F5010155515B2756515C23E86A5D2305
:100C20000E2E1BEF06F05CC157F15DC158F15B6BF6
:100C30005C6B5D6B078E0201002FE5EF07F03C0E49
:100C4000006F00C10CF101C10DF102C10EF103C131
:100C50000FF104C110F105C111F106C112F107C174
:100C600013F108C114F109C115F10AC116F10BC144
:100C700017F134C135F105012F51000AD8B4E4EF62
:100C800006F005012F51010AD8B46EEF06F00501F8
:100C90002F51020AD8B4AFEF06F005012F51030A15
:100CA000D8B4AFEF06F005012F51040AD8B4AFEF66
:100CB00006F005012F51050AD8B4AFEF06F0050183
:100CC0002F51060AD8B4AFEF06F005012F51070ADD
:100CD000D8B4AFEF06F02F6BE4EF06F005015367D1
:100CE00079EF06F0546779EF06F0556779EF06F073
:100CF00056677DEF06F0E4EF06F057C500F158C5E2
:100D000001F159C502F15AC503F10101010E046F49
:100D1000000E056F000E066F000E076FBFEC25F08A
:100D200000C157F501C158F502C159F503C15AF583
:100D30000067A2EF06F00167A2EF06F00267A2EFDC
:100D400006F00367E4EF06F053C557F554C558F5B0
:100D500055C559F556C55AF50F88E4EF06F005015B
:100D60003067B5EF06F0E4EF06F00FBECAEF06F00D
:100D700010A0CFEF06F001014767C6EF06F0486705
:100D8000C6EF06F04967C6EF06F04A67CAEF06F0FD
:100D9000CFEF06F007AECFEF06F0E1EF06F005016A
:100DA000312FE4EF06F03C0E316F302FE4EF06F008
:100DB0000101000E626FE00E636FA50E646F010EFD
:100DC000656F0501306B0F880501626B33B7EAEF81
:100DD00006F062810CC100F10DC101F10EC102F1FA
:100DE0000FC103F110C104F111C105F112C106F1E7
:100DF00013C107F114C108F115C109F116C10AF1B7
:100E000017C10BF135C134F100C10CF101C10DF175
:100E100002C10EF103C10FF104C110F105C111F1BE
:100E200006C112F107C113F108C114F109C115F18E
:100E30000AC116F10BC117F134C135F101018A67FE
:100E400029EF07F08B6729EF07F08C6729EF07F090
:100E50008D672DEF07F05DEF07F08EC100F18FC1B8
:100E600001F190C102F191C103F10101010E046F82
:100E7000000E056F000E066F000E076FBFEC25F029
:100E800000C18EF101C18FF102C190F103C191F156
:100E9000006752EF07F0016752EF07F0026752EF69
:100EA00007F003675DEF07F08AC18EF18BC18FF108
:100EB0008CC190F18DC191F10F80D57ED5BE69D0E6
:100EC000D6CF47F1D7CF48F145C149F1E86AE8CF1D
:100ED0004AF1109047C100F148C101F149C102F146
:100EE0004AC103F101010A0E046F000E056F000EE6
:100EF000066F000E076FBFEC25F003AF10800101F5
:100F000054A78FEF07F00F9A0F9C0F9E0101000E60
:100F10005E6F600E5F6F3D0E606F080E616F0101C6
:100F200047BF9FEF07F048679FEF07F049679FEFC4
:100F300007F04A679FEF07F0F288C4EF07F0F298D6
:100F40005E6B5F6B606B616B966B976B986B996B6D
:100F50009A6B9B6B9C6B9D6B9E6B9F6BA06BA16B4D
:100F6000A26BA36BA46BA56BA66BA76BA86BA96BFD
:100F7000AA6BAB6BAC6BAD6BAE6BAF6BB06BB16BAD
:100F8000B26BB36BB46BB56BD76AD66A0101456BB4
:100F9000466B0CC100F10DC101F10EC102F10FC190
:100FA00003F110C104F111C105F112C106F113C121
:100FB00007F114C108F115C109F116C10AF117C1F1
:100FC0000BF135C134F1E5EF07F002C0E0FF00504E
:100FD00001C0D8FF1000A6B2EBEF07F00CC0A9FFCC
:100FE0000BC0A8FFA69EA69CA684F29E550EA76ED7
:100FF000AA0EA76EA682F28EA694A6B2FDEF07F007
:101000000C2A1200A96EA69EA69CA680A8500C2AA7
:10101000120004012C0E826FF8EC0AF0BAEC26F0F4
:101020000C5002EC08F0E8CF00F10C5002EC08F094
:10103000E8CF01F101AF22EF08F00101FF0E026FCE
:10104000FF0E036F5DEC26F029672EEF08F0040118
:10105000200E826FF8EC0AF033EF08F004012D0E39
:10106000826FF8EC0AF087EC24F01200076A0F6A2E
:10107000106A0F010D0EC16E860EC06E030EC26E99
:101080000F01680E896E130E926E080E8A6E8A6AC0
:10109000F30E936E8B6A900E946EF18EF19E0E6A33
:1010A00001015B6B5C6B5D6B576B586BF29A0101D6
:1010B000476B486B496B4A6B4B6B4C6B4D6B4E6B84
:1010C0004F6B506B516B526B456B466BD76AD66A50
:1010D0000F01280ED56EF28A9D90B00ECD6E0101E3
:1010E0005E6B5F6B606B616B626B636B646B656B9C
:1010F000666B676B686B696B536B546BCF6ACE6AB8
:101100000F9A0F9C0F9E9D80760ECA6E9D820201E3
:101110003C0E006FCC6A160E02EC08F0E8CF00F12E
:10112000170E02EC08F0E8CF01F1180E02EC08F0FF
:10113000E8CF02F1190E02EC08F0E8CF03F101014B
:1011400003AFBDEF08F0BAEC26F0160E0C6E00C12E
:101150000BF0EBEC07F0170E0C6E01C10BF0EBEC93
:1011600007F0180E0C6E02C10BF0EBEC07F0190E35
:101170000C6E03C10BF0EBEC07F000C18AF101C16A
:101180008BF102C18CF103C18DF100C18EF101C15F
:101190008FF102C190F103C191F11A0E02EC08F037
:1011A000E8CF00F11B0E02EC08F0E8CF01F11C0EB5
:1011B00002EC08F0E8CF02F11D0E02EC08F0E8CFD7
:1011C00003F1010103AF13EF09F0BAEC26F01A0E98
:1011D0000C6E00C10BF0EBEC07F01B0E0C6E01C1A6
:1011E0000BF0EBEC07F01C0E0C6E02C10BF0EBECFD
:1011F00007F01D0E0C6E03C10BF0EBEC07F01A0E9E
:1012000002EC08F0E8CF00F11B0E02EC08F0E8CF8A
:1012100001F11C0E02EC08F0E8CF02F11D0E02EC09
:1012200008F0E8CF03F100C192F101C193F102C1CE
:1012300094F103C195F1240EAC6E900EAB6E240EAA
:10124000AC6E080EB86E000EB06E1F0EAF6E0401CD
:10125000806B816B0F01900EAB6E0F019D8A0301B5
:10126000806B816BC26B8B9249EC2DF049EC2DF0B9
:1012700079EC30F02AEC2BF0200E02EC08F0E8CFED
:101280002FF505012F51FF0AD8A44EEF09F02F6B5F
:10129000200E0C6E2FC50BF0EBEC07F00501010ED4
:1012A000306F3C0E316F250E02EC08F0E8CF00F1F4
:1012B000260E02EC08F0E8CF01F1270E02EC08F050
:1012C000E8CF02F1280E02EC08F0E8CF03F10101AB
:1012D00003AF85EF09F0BAEC26F0250E0C6E00C1C5
:1012E0000BF0EBEC07F0260E0C6E01C10BF0EBECF3
:1012F00007F0270E0C6E02C10BF0EBEC07F0280E86
:101300000C6E03C10BF0EBEC07F000C153F501C10B
:1013100054F502C155F503C156F500C157F501C199
:1013200058F502C159F503C15AF5290E02EC08F02F
:10133000E8CF5BF505015C515B5DD8A05BC55CF552
:1013400005012F51020A0EE181B8B2EF09F0050143
:101350005C2FAFEF09F05BC55CF5B2EF09F081BA25
:10136000B8EF30F0210E02EC08F0E8CF00F1220EC9
:1013700002EC08F0E8CF01F1230E02EC08F0E8CF10
:1013800002F1240E02EC08F0E8CF03F1010103AFF3
:10139000F8EF09F0BAEC26F0210E0C6E00C10BF04C
:1013A000EBEC07F0220E0C6E01C10BF0EBEC07F03A
:1013B000230E0C6E02C10BF0EBEC07F0240E0C6E4A
:1013C00003C10BF0EBEC07F0210E02EC08F0E8CFC4
:1013D00000F1220E02EC08F0E8CF01F1230E02EC3E
:1013E00008F0E8CF02F1240E02EC08F0E8CF03F198
:1013F00000C15DF501C15EF502C15FF503C160F595
:1014000061EC2AF023EC29F073EC28F005012F5150
:10141000030A12E005012F51040A1DE005012F51B6
:10142000050A24E005012F51060A32E005012F517B
:10143000070A38E05BEF0AF0ACC500F101010F0EBE
:10144000001701010051000A36E001010051050AB0
:1014500032E058EF0AF0ACC500F101010F0E0017A1
:1014600001010051000A27E058EF0AF00501AC51D4
:10147000000A21E00501AC51150A1DE00501AC513F
:10148000300A19E00501AC51450A15E058EF0AF0A1
:101490000501AC51000A0FE00501AC51300A0BE028
:1014A00058EF0AF00501AC51000A05E058EF0AF0C8
:1014B00081BAB8EF30F01EEC28F007900001F28EF0
:1014C000F28C07B008EF23F00FB0E9EF1DF00FB872
:1014D000ADEF17F00301805181197F0BD8B408EFED
:1014E00023F013EE00F081517F0BE126812BE7CF33
:1014F000E8FFE00BD8B408EF23F023EE82F0C251EE
:101500003F0BD926E7CFDFFFC22BDF50780AD8A4E4
:1015100008EF23F007808EC100F18FC101F190C167
:1015200002F191C103F10101040E046F000E056F79
:10153000000E066F000E076FBFEC25F000AFAAEF9C
:101540000AF00101030E8E6F000E8F6F000E906F78
:10155000000E916F03018251720AD8B4E9EF1DF0B9
:101560008251520AD8B4E9EF1DF08251750AD8B4FD
:10157000E9EF1DF08251630AD8B4C4EF1FF0825125
:10158000690AD8B4A4EF1AF082517A0AD8B4B7EF36
:101590001BF08251490AD8B443EF1AF08251500A25
:1015A000D8B461EF19F08251700AD8B4A4EF19F0E1
:1015B0008251540AD8B4CFEF19F08251740AD8B4CA
:1015C00015EF1AF08251730AD8B419EF1DF0825149
:1015D000530AD8B47EEF1DF082514C0AD8B45CEFA8
:1015E00010F08251760AD8B40CEF0BF0F9EF1FF02F
:1015F000040114EE00F080517F0BE12682C4E7FF66
:10160000802B120004010D0E826FF8EC0AF00A0E16
:10161000826FF8EC0AF0120003018351300AD8B44B
:101620002DEF0BF003018351310AD8B464EF0BF0B6
:1016300003018351320AD8B419EF0DF0030183512D
:10164000330AD8B4CEEF0EF003018351340AD8B474
:1016500074EF0FF0D8A4F9EF1FF00401760E826F3B
:10166000F8EC0AF00401300E826FF8EC0AF0040185
:101670002C0E826FF8EC0AF028EC27F0BAEC26F07A
:1016800000C600F101C601F15DEC26F030C182F424
:101690000401300E8227F8EC0AF031C182F4040113
:1016A000300E8227F8EC0AF032C182F40401300EC9
:1016B0008227F8EC0AF033C182F40401300E82274D
:1016C000F8EC0AF00EEF18F00401760E826FF8ECD9
:1016D0000AF00401310E826FF8EC0AF00784010170
:1016E000036B026B02C600F103C601F101AF7DEF8F
:1016F0000BF0FF0E026FFF0E036F0101076B066B0D
:1017000004C604F105C605F105AF8BEF0BF0FF0E23
:10171000066FFF0E076FC4EC25F00101076B066B27
:1017200006C604F107C605F105AF9BEF0BF0FF0EEF
:10173000066FFF0E076FC4EC25F00101076B066B07
:1017400008C604F109C605F105AFABEF0BF0FF0EBB
:10175000066FFF0E076FC4EC25F0D890010103332C
:10176000023301330033D8900101033302330133D4
:10177000003304012C0E826FF8EC0AF00101036BB8
:10178000026B01C101F100C100F101AFCDEF0BF01F
:101790000101FF0E026FFF0E036F5DEC26F029675B
:1017A000D4EF0BF0D9EF0BF004012D0E826FF8ECA3
:1017B0000AF02FC182F40401300E8227F8EC0AF0FF
:1017C00030C182F40401300E8227F8EC0AF031C1F6
:1017D00082F40401300E8227F8EC0AF032C182F460
:1017E0000401300E8227F8EC0AF033C182F40401C0
:1017F000300E8227F8EC0AF00101036B026B0AC677
:1018000000F10BC601F101AF0AEF0CF0FF0E026F01
:10181000FF0E036F0101076B066B0CC604F10DC6CA
:1018200005F105AF18EF0CF0FF0E066FFF0E076F06
:10183000C4EC25F00101076B066B0EC604F10FC660
:1018400005F105AF28EF0CF0FF0E066FFF0E076FD6
:10185000C4EC25F00101076B066B10C604F111C63C
:1018600005F105AF38EF0CF0FF0E066FFF0E076FA6
:10187000C4EC25F0D8900101033302330133003367
:10188000D8900101033302330133003304012C0EDD
:10189000826FF8EC0AF00101036B026B01C101F1E8
:1018A00000C100F101AF5AEF0CF00101FF0E026F11
:1018B000FF0E036F5DEC26F0296761EF0CF066EF19
:1018C0000CF004012D0E826FF8EC0AF02FC182F4A7
:1018D0000401300E8227F8EC0AF030C182F40401D2
:1018E000300E8227F8EC0AF031C182F40401300E88
:1018F0008227F8EC0AF032C182F40401300E82270C
:10190000F8EC0AF033C182F40401300E8227F8ECBF
:101910000AF00101036B026B12C600F113C601F15C
:1019200001AF97EF0CF0FF0E026FFF0E036F010186
:10193000076B066B14C604F115C605F105AFA5EFDC
:101940000CF0FF0E066FFF0E076FC4EC25F00101CF
:10195000076B066B16C604F117C605F105AFB5EFA8
:101960000CF0FF0E066FFF0E076FC4EC25F00101AF
:10197000076B066B18C604F119C605F105AFC5EF74
:101980000CF0FF0E066FFF0E076FC4EC25F0D89029
:1019900001010333023301330033D89001010333D3
:1019A00002330133003304012C0E826FF8EC0AF08D
:1019B0000101036B026B01C101F100C100F101AF34
:1019C000E7EF0CF00101FF0E026FFF0E036F5DECFD
:1019D00026F02967EEEF0CF0F3EF0CF004012D0E6A
:1019E000826FF8EC0AF02FC182F40401300E8227D6
:1019F000F8EC0AF030C182F40401300E8227F8ECD2
:101A00000AF031C182F40401300E8227F8EC0AF0AA
:101A100032C182F40401300E8227F8EC0AF033C19F
:101A200082F40401300E8227F8EC0AF007940EEFDE
:101A300018F00401760E826FF8EC0AF00401320E01
:101A4000826FF8EC0AF007840101036B026B1AC67F
:101A500000F11BC601F101AF32EF0DF0FF0E026F76
:101A6000FF0E036F0101076B066B1CC604F11DC658
:101A700005F105AF40EF0DF0FF0E066FFF0E076F8B
:101A8000C4EC25F00101076B066B1EC604F11FC6EE
:101A900005F105AF50EF0DF0FF0E066FFF0E076F5B
:101AA000C4EC25F00101076B066B20C604F121C6CA
:101AB00005F105AF60EF0DF0FF0E066FFF0E076F2B
:101AC000C4EC25F0D8900101033302330133003315
:101AD000D8900101033302330133003304012C0E8B
:101AE000826FF8EC0AF00101036B026B01C101F196
:101AF00000C100F101AF82EF0DF00101FF0E026F96
:101B0000FF0E036F5DEC26F0296789EF0DF08EEF75
:101B10000DF004012D0E826FF8EC0AF02FC182F453
:101B20000401300E8227F8EC0AF030C182F404017F
:101B3000300E8227F8EC0AF031C182F40401300E35
:101B40008227F8EC0AF032C182F40401300E8227B9
:101B5000F8EC0AF033C182F40401300E8227F8EC6D
:101B60000AF00101036B026B22C600F123C601F1EA
:101B700001AFBFEF0DF0FF0E026FFF0E036F01010B
:101B8000076B066B24C604F125C605F105AFCDEF42
:101B90000DF0FF0E066FFF0E076FC4EC25F001017C
:101BA000076B066B26C604F127C605F105AFDDEF0E
:101BB0000DF0FF0E066FFF0E076FC4EC25F001015C
:101BC000076B066B28C604F129C605F105AFEDEFDA
:101BD0000DF0FF0E066FFF0E076FC4EC25F0D890D6
:101BE00001010333023301330033D8900101033381
:101BF00002330133003304012C0E826FF8EC0AF03B
:101C00000101036B026B01C101F100C100F101AFE1
:101C10000FEF0EF00101FF0E026FFF0E036F5DEC80
:101C200026F0296716EF0EF01BEF0EF004012D0EC3
:101C3000826FF8EC0AF02FC182F40401300E822783
:101C4000F8EC0AF030C182F40401300E8227F8EC7F
:101C50000AF031C182F40401300E8227F8EC0AF058
:101C600032C182F40401300E8227F8EC0AF033C14D
:101C700082F40401300E8227F8EC0AF00101036BB4
:101C8000026B2AC600F12BC601F101AF4CEF0EF03A
:101C9000FF0E026FFF0E036F0101076B066B2CC670
:101CA00004F12DC605F105AF5AEF0EF0FF0E066FD9
:101CB000FF0E076FC4EC25F00101076B066B2EC603
:101CC00004F12FC605F105AF6AEF0EF0FF0E066FA7
:101CD000FF0E076FC4EC25F00101076B066B30C6E1
:101CE00004F131C605F105AF7AEF0EF0FF0E066F75
:101CF000FF0E076FC4EC25F0D890010103330233C7
:101D000001330033D8900101033302330133003330
:101D100004012C0E826FF8EC0AF00101036B026BD8
:101D200001C101F100C100F101AF9CEF0EF0010112
:101D3000FF0E026FFF0E036F5DEC26F02967A3EF25
:101D40000EF0A8EF0EF004012D0E826FF8EC0AF0F1
:101D50002FC182F40401300E8227F8EC0AF030C162
:101D600082F40401300E8227F8EC0AF031C182F4CB
:101D70000401300E8227F8EC0AF032C182F404012B
:101D8000300E8227F8EC0AF033C182F40401300EE1
:101D90008227F8EC0AF007940EEF18F00401760E93
:101DA000826FF8EC0AF00401330E826FF8EC0AF04F
:101DB00004012C0E826FF8EC0AF085C382F4F8EC73
:101DC0000AF0640E0D6E03018551320A02E16A0EBB
:101DD0000D6E03018551330A02E1700E0D6E030191
:101DE0008551340A02E1760E0D6E03018551350AE4
:101DF00002E17C0E0D6E03018551360A02E1820E6E
:101E00000D6E03018651780A65E00DC00CF0FBEC05
:101E100026F02981030187512D0AD8B412EF0FF063
:101E20000101299188C32FF189C330F18AC331F1AF
:101E30008BC332F18CC333F108EC27F07FEC26F032
:101E400000C10BF0EBEC07F001C10BF0EBEC07F07D
:101E5000FBEC26F0298103018E512D0AD8B433EF13
:101E60000FF0010129918FC32FF190C330F191C37D
:101E700031F192C332F193C333F108EC27F07FECD8
:101E800026F000C10BF0EBEC07F001C10BF0EBEC1E
:101E900007F0FBEC26F02981030195512D0AD8B4F7
:101EA00054EF0FF00101299196C32FF197C330F140
:101EB00098C331F199C332F19AC333F108EC27F09A
:101EC0007FEC26F000C10BF0EBEC07F001C10BF04A
:101ED000EBEC07F00DC00CF009EC08F009EC08F091
:101EE00009EC08F00EEF18F00401760E826FF8ECA2
:101EF0000AF00401340E826FF8EC0AF003018451F9
:101F0000780AD8B44CEF10F03E0E0C6EFBEC26F0C5
:101F10002981030185512D0AD8B491EF0FF00101F9
:101F2000299186C32FF187C330F188C331F189C36A
:101F300032F18AC333F108EC27F07FEC26F000C1C0
:101F40000BF0EBEC07F001C10BF0EBEC07F0FBEC56
:101F500026F0298103018C512D0AD8B4B2EF0FF07D
:101F6000010129918DC32FF18EC330F18FC331F15F
:101F700090C332F191C333F108EC27F07FEC26F0E7
:101F800000C10BF0EBEC07F001C10BF0EBEC07F03C
:101F9000FBEC26F02981030193512D0AD8B4D3EF2D
:101FA0000FF00101299194C32FF195C330F196C32D
:101FB00031F197C332F198C333F108EC27F07FEC8D
:101FC00026F000C10BF0EBEC07F001C10BF0EBECDD
:101FD00007F0FBEC26F0298103019A512D0AD8B4B1
:101FE000F4EF0FF0010129919BC32FF19CC330F155
:101FF0009DC331F19EC332F19FC333F108EC27F04A
:102000007FEC26F000C10BF0EBEC07F001C10BF008
:10201000EBEC07F0FBEC26F029810301A1512D0A1E
:10202000D8B415EF10F001012991A2C32FF1A3C379
:1020300030F1A4C331F1A5C332F1A6C333F108ECEA
:1020400027F07FEC26F000C10BF0EBEC07F001C1AC
:102050000BF0EBEC07F0FBEC26F029810301A85113
:102060002D0AD8B436EF10F001012991A9C32FF140
:10207000AAC330F1ABC331F1ACC332F1ADC333F11C
:1020800008EC27F07FEC26F000C10BF0EBEC07F03A
:1020900001C10BF0EBEC07F03E0E0C6E09EC08F002
:1020A00009EC08F009EC08F009EC08F009EC08F07C
:1020B00009EC08F00EEF18F003018351300AD8B490
:1020C0001DEF13F003018351310AD8B429EF14F046
:1020D00003018351320AD8B495EF14F00301835100
:1020E000330AD8B4A3EF14F003018351340AD8B4EF
:1020F000B1EF14F003018351350AD8B4B2EF17F0F1
:1021000003018351360AD8B4E0EF17F0030183517D
:10211000460AD8B406EF17F0030183514D0AD8B42C
:1021200096EF11F0030183516D0AD8B4B0EF11F0AE
:10213000030183515A0AD8B4A3EF13F0030183516A
:10214000490AD8B4E0EF18F003018351500AD8B41B
:1021500012EF18F003018351540AD8B48BEF18F032
:1021600003018351630AD8B4D0EF11F00301835106
:10217000430AD8B4C8EF12F003018351730AD8B4EC
:10218000CEEF11F003018351610AD8B4E3EF10F0F0
:1021900003018351650AD8B46BEF13F00301835137
:1021A000450AD8B479EF13F003018351620AD8B419
:1021B00087EF13F003018351420AD8B495EF13F06F
:1021C000D8A4F9EF1FF004014C0E826FF8EC0AF06E
:1021D0000401610E826FF8EC0AF023EC29F004018F
:1021E0002C0E826FF8EC0AF0BAEC26F0ABC500F1C9
:1021F00001015DEC26F031C182F40401300E82272A
:10220000F8EC0AF032C182F40401300E8227F8ECB7
:102210000AF033C182F40401300E8227F8EC0AF090
:1022200004012C0E826FF8EC0AF0BAEC26F0ACC573
:1022300000F101015DEC26F031C182F40401300EA1
:102240008227F8EC0AF032C182F40401300E8227B2
:10225000F8EC0AF033C182F40401300E8227F8EC66
:102260000AF004012C0E826FF8EC0AF0BAEC26F0AA
:10227000ADC500F101015DEC26F031C182F404012D
:10228000300E8227F8EC0AF032C182F40401300EDD
:102290008227F8EC0AF033C182F40401300E822761
:1022A000F8EC0AF004012C0E826FF8EC0AF0BAEC9C
:1022B00026F0AEC500F101015DEC26F031C182F4DB
:1022C0000401300E8227F8EC0AF032C182F40401D6
:1022D000300E8227F8EC0AF033C182F40401300E8C
:1022E0008227F8EC0AF004012C0E826FF8EC0AF059
:1022F000BAEC26F0B3C500F101015DEC26F031C166
:1023000082F40401300E8227F8EC0AF032C182F424
:102310000401300E8227F8EC0AF033C182F4040184
:10232000300E8227F8EC0AF00EEF18F0FBEC26F0E6
:1023300084C333F108EC27F07FEC26F0200E0C6EFE
:1023400000C10BF0EBEC07F000C12FF505012F5198
:10235000000A06E005012F51010A02E0C9EC29F04C
:1023600004014C0E826FF8EC0AF004014D0E826FEE
:10237000F8EC0AF004012C0E826FF8EC0AF0BAECCB
:1023800026F02FC500F15DEC26F033C182F4040184
:10239000300E8227F8EC0AF00EEF18F0B8EF30F0AC
:1023A00004014C0E826FF8EC0AF00401630E826F98
:1023B000F8EC0AF073EC28F004012C0E826FF8ECB4
:1023C0000AF0E5EC11F00EEF18F0BAEC26F0B1C50A
:1023D00000F10101003B0F0E00175DEC26F033C148
:1023E00082F40401300E8227F8EC0AF0B1C500F146
:1023F00001010F0E010100175DEC26F033C182F4DC
:102400000401300E8227F8EC0AF004012D0E826FD1
:10241000F8EC0AF0B0C500F10101003B0F0E001707
:102420005DEC26F033C182F40401300E8227F8EC13
:102430000AF0B0C500F101010F0E010100175DECBB
:1024400026F033C182F40401300E8227F8EC0AF042
:1024500004012D0E826FF8EC0AF0AFC500F1010106
:10246000003B0F0E00175DEC26F033C182F404012F
:10247000300E8227F8EC0AF0AFC500F101010F0E13
:10248000010100175DEC26F033C182F40401300E27
:102490008227F8EC0AF00401200E826FF8EC0AF0B3
:1024A000AEC500F10F0E010100175DEC26F033C13F
:1024B00082F40401300E8227F8EC0AF00401200EA9
:1024C000826FF8EC0AF0ADC500F101010101003B9B
:1024D0000F0E00175DEC26F033C182F40401300EBC
:1024E0008227F8EC0AF0ADC500F101010F0E0101E1
:1024F00000175DEC26F033C182F40401300E822710
:10250000F8EC0AF004013A0E826FF8EC0AF0ACC560
:1025100000F10101003B0F0E00175DEC26F033C106
:1025200082F40401300E8227F8EC0AF0ACC500F109
:1025300001010F0E010100175DEC26F033C182F49A
:102540000401300E8227F8EC0AF004013A0E826F83
:10255000F8EC0AF0ABC500F10101003B0F0E0017CB
:102560005DEC26F033C182F40401300E8227F8ECD2
:102570000AF0ABC500F101010F0E00175DEC26F06B
:1025800033C182F40401300E8227F8EC0AF0120005
:1025900084C3E8FF0F0BE83AE8CFB1F585C3E8FF45
:1025A0000F0B0501B11387C3E8FF0F0BE83AE8CF23
:1025B000B0F588C3E8FF0F0B0501B0138AC3E8FF2D
:1025C0000F0BE83AE8CFAFF58BC3E8FF0F0B05011F
:1025D000AF138DC3E8FF0F0BE8CFAEF58FC3E8FF55
:1025E0000F0BE83AE8CFADF590C3E8FF0F0B0501FC
:1025F000AD1392C3E8FF0F0BE83AE8CFACF593C3F5
:10260000E8FF0F0B0501AC1395C3E8FF0F0BE83A89
:10261000E8CFABF596C3E8FF0F0B0501AB13D2EC87
:1026200028F004014C0E826FF8EC0AF00401430E0E
:10263000826FF8EC0AF0DAEF11F079EC30F0BAECD6
:1026400026F02DC500F15DEC26F004014C0E826FE2
:10265000F8EC0AF00401300E826FF8EC0AF0040185
:102660002C0E826FF8EC0AF031C182F40401300EB6
:102670008227F8EC0AF032C182F40401300E82277E
:10268000F8EC0AF033C182F40401300E8227F8EC32
:102690000AF004012C0E826FF8EC0AF0BAEC26F076
:1026A0002EC500F15DEC26F031C182F40401300E3C
:1026B0008227F8EC0AF032C182F40401300E82273E
:1026C000F8EC0AF033C182F40401300E8227F8ECF2
:1026D0000AF00EEF18F004014C0E826FF8EC0AF0CD
:1026E0000401650E826FF8EC0AF0B2EC2AF00EEFEE
:1026F00018F004014C0E826FF8EC0AF00401450E4C
:10270000826FF8EC0AF0CFEC2AF00EEF18F004011B
:102710004C0E826FF8EC0AF00401620E826FF8EC46
:102720000AF009EC2BF00EEF18F004014C0E826F4A
:10273000F8EC0AF00401420E826FF8EC0AF0ECECBF
:102740002AF00EEF18F004014C0E826FF8EC0AF03C
:1027500004015A0E826FF8EC0AF004012C0E826F0D
:10276000F8EC0AF079EC30F0BAEC26F005012E51C5
:10277000130A06E005012E51170A0DE0D4EF13F0FD
:102780000101000E006F000E016F100E026F000EAF
:10279000036FD4EF13F00101000E006F000E016F04
:1027A000000E026F010E036F0101100E046F000E88
:1027B000056F000E066F000E076FF0EC25F05DEC64
:1027C00026F02AC182F40401300E8227F8EC0AF0C8
:1027D0002BC182F40401300E8227F8EC0AF02CC1E0
:1027E00082F40401300E8227F8EC0AF02DC182F445
:1027F0000401300E8227F8EC0AF02EC182F40401A5
:10280000300E8227F8EC0AF02FC182F40401300E5A
:102810008227F8EC0AF030C182F40401300E8227DE
:10282000F8EC0AF031C182F40401300E8227F8EC92
:102830000AF032C182F40401300E8227F8EC0AF06B
:1028400033C182F40401300E8227F8EC0AF00EEF57
:1028500018F004014C0E826FF8EC0AF00401310EFE
:10286000826FF8EC0AF004012C0E826FF8EC0AF08B
:1028700025C500F126C501F127C502F128C503F1E0
:102880000101200E046F000E056F000E066F000E92
:10289000076FF0EC25F05DEC26F02AC182F404010C
:1028A000300E8227F8EC0AF02BC182F40401300EBE
:1028B0008227F8EC0AF02CC182F40401300E822742
:1028C000F8EC0AF02DC182F40401300E8227F8ECF6
:1028D0000AF02EC182F40401300E8227F8EC0AF0CF
:1028E0002FC182F40401300E8227F8EC0AF030C1C7
:1028F00082F40401300E8227F8EC0AF031C182F430
:102900000401300E8227F8EC0AF032C182F404018F
:10291000300E8227F8EC0AF033C182F40401300E45
:102920008227F8EC0AF00EEF18F004014C0E826FCB
:10293000F8EC0AF00401320E826FF8EC0AF0FFECBA
:102940002CF00EEF18F004014C0E826FF8EC0AF038
:102950000401330E826FF8EC0AF05CEC2DF033EFDB
:1029600014F004014C0E826FF8EC0AF00401340EEE
:10297000826FF8EC0AF004012C0E826FF8EC0AF07A
:10298000FBEC26F084C32AF185C32BF186C32CF11E
:1029900087C32DF188C32EF189C32FF18AC330F18B
:1029A0008BC331F18CC332F18DC333F10101296B3B
:1029B00008EC27F07FEC26F0200E046F000E056F68
:1029C000000E066F000E076FD0EC25F000C121F558
:1029D00001C122F502C123F503C124F52CEC30F02E
:1029E00034C5ABF535C5ACF536C5ADF537C5AEF577
:1029F00038C5AFF539C5B0F53AC5B1F5E5EC11F01C
:102A000004012C0E826FF8EC0AF03BC500F13CC5C6
:102A100001F13DC502F13EC503F10101000E046F55
:102A2000000E056F010E066F000E076FF0EC25F02B
:102A30005DEC26F029671FEF15F024EF15F0040177
:102A40002D0E826FF8EC0AF030C182F40401300ED2
:102A50008227F8EC0AF031C182F40401300E82279B
:102A6000F8EC0AF004012E0E826FF8EC0AF032C185
:102A700082F40401300E8227F8EC0AF033C182F4AC
:102A80000401300E8227F8EC0AF004012C0E826F4C
:102A9000F8EC0AF0BAEC26F03FC500F140C501F1B0
:102AA00023EC21F004012C0E826FF8EC0AF0BAEC52
:102AB00026F041C500F15DEC26F031C182F404013D
:102AC000300E8227F8EC0AF032C182F40401300E95
:102AD0008227F8EC0AF033C182F40401300E822719
:102AE000F8EC0AF004012C0E826FF8EC0AF00101F8
:102AF000036B026B48C501F147C500F101AF86EFDA
:102B000015F00101FF0E026FFF0E036F5DEC26F062
:102B100029678DEF15F092EF15F004012D0E826FED
:102B2000F8EC0AF02FC182F40401300E8227F8EC91
:102B30000AF030C182F40401300E8227F8EC0AF06A
:102B400031C182F40401300E8227F8EC0AF032C160
:102B500082F40401300E8227F8EC0AF033C182F4CB
:102B60000401300E8227F8EC0AF004012C0E826F6B
:102B7000F8EC0AF00101036B026B4AC501F149C58B
:102B800000F101AFC9EF15F00101FF0E026FFF0E5A
:102B9000036F5DEC26F02967D0EF15F0D5EF15F047
:102BA00004012D0E826FF8EC0AF02FC182F40401AB
:102BB000300E8227F8EC0AF030C182F40401300EA6
:102BC0008227F8EC0AF031C182F40401300E82272A
:102BD000F8EC0AF032C182F40401300E8227F8ECDE
:102BE0000AF033C182F40401300E8227F8EC0AF0B7
:102BF00004012C0E826FF8EC0AF00101036B026BEA
:102C00004CC501F14BC500F101AF0CEF16F001010D
:102C1000FF0E026FFF0E036F5DEC26F0296713EFC6
:102C200016F018EF16F004012D0E826FF8EC0AF082
:102C30002FC182F40401300E8227F8EC0AF030C173
:102C400082F40401300E8227F8EC0AF031C182F4DC
:102C50000401300E8227F8EC0AF032C182F404013C
:102C6000300E8227F8EC0AF033C182F40401300EF2
:102C70008227F8EC0AF004012C0E826FF8EC0AF0BF
:102C80000101036B026B4EC501F14DC500F101AFAF
:102C90004FEF16F00101FF0E026FFF0E036F5DECA8
:102CA00026F0296756EF16F05BEF16F004012D0EA3
:102CB000826FF8EC0AF02FC182F40401300E8227F3
:102CC000F8EC0AF030C182F40401300E8227F8ECEF
:102CD0000AF031C182F40401300E8227F8EC0AF0C8
:102CE00032C182F40401300E8227F8EC0AF033C1BD
:102CF00082F40401300E8227F8EC0AF004012C0E55
:102D0000826FF8EC0AF00101036B026B50C501F110
:102D10004FC500F101AF92EF16F00101FF0E026FF7
:102D2000FF0E036F5DEC26F0296799EF16F09EEF1A
:102D300016F004012D0E826FF8EC0AF02FC182F418
:102D40000401300E8227F8EC0AF030C182F404014D
:102D5000300E8227F8EC0AF031C182F40401300E03
:102D60008227F8EC0AF032C182F40401300E822787
:102D7000F8EC0AF033C182F40401300E8227F8EC3B
:102D80000AF004012C0E826FF8EC0AF00101036BCB
:102D9000026B52C501F151C500F101AFD5EF16F03C
:102DA0000101FF0E026FFF0E036F5DEC26F0296735
:102DB000DCEF16F0E1EF16F004012D0E826FF8EC57
:102DC0000AF02FC182F40401300E8227F8EC0AF0D9
:102DD00030C182F40401300E8227F8EC0AF031C1D0
:102DE00082F40401300E8227F8EC0AF032C182F43A
:102DF0000401300E8227F8EC0AF033C182F404019A
:102E0000300E8227F8EC0AF00EEF18F0FBEC26F0FB
:102E100085C32AF186C32BF187C32CF188C32DF11A
:102E200089C32EF18AC32FF18BC330F18CC331F1EA
:102E30008DC332F18EC333F10101296B08EC27F009
:102E40007FEC26F00101010E046F000E056F000EED
:102E5000066F000E076FBFEC25F0100E046F000E1A
:102E6000056F000E066F000E076FD0EC25F000C155
:102E700029F501C12AF502C12BF503C12CF588EC17
:102E80002CF004014C0E826FF8EC0AF00401460E9F
:102E9000826FF8EC0AF004012C0E826FF8EC0AF055
:102EA00025C500F126C501F127C502F128C503F1AA
:102EB0000101100E046F000E056F000E066F000E6C
:102EC000076FF0EC25F05DEC26F02AC182F40401D6
:102ED000300E8227F8EC0AF02BC182F40401300E88
:102EE0008227F8EC0AF02CC182F40401300E82270C
:102EF000F8EC0AF02DC182F40401300E8227F8ECC0
:102F00000AF02EC182F40401300E8227F8EC0AF098
:102F10002FC182F40401300E8227F8EC0AF030C190
:102F200082F40401300E8227F8EC0AF031C182F4F9
:102F30000401300E8227F8EC0AF032C182F4040159
:102F4000300E8227F8EC0AF033C182F40401300E0F
:102F50008227F8EC0AF00EEF18F00F985CEC2DF0D9
:102F60000EEF18F004014C0E826FF8EC0AF0040129
:102F7000350E826FF8EC0AF004012C0E826FF8EC2B
:102F80000AF0BAEC26F00784B5C500F107945DECB1
:102F900026F031C182F40401300E8227F8EC0AF0E9
:102FA00032C182F40401300E8227F8EC0AF033C1FA
:102FB00082F40401300E8227F8EC0AF00EEF18F0CC
:102FC0001FEC2DF0BAEC26F033C500F15DEC26F0D5
:102FD00004014C0E826FF8EC0AF00401360E826F89
:102FE000F8EC0AF004012C0E826FF8EC0AF031C103
:102FF00082F40401300E8227F8EC0AF032C182F428
:103000000401300E8227F8EC0AF033C182F4040187
:10301000300E8227F8EC0AF00EEF18F002EC0BF0FD
:10302000F9EF1FF004014C0E826FF8EC0AF0040176
:10303000500E826FF8EC0AF004012C0E826FF8EC4F
:103040000AF085C32AF186C32BF187C32CF188C30C
:103050002DF189C32EF18AC32FF18BC330F18CC3BC
:1030600031F18DC332F18EC333F1010108EC27F049
:103070007FEC26F003018451530A0DE003018451D3
:103080004D0A38E00401780E826FF8EC0AF002EC89
:103090000BF0F9EF1FF00401530E826FF8EC0AF009
:1030A000250E0C6E00C10BF0EBEC07F0260E0C6E3B
:1030B00001C10BF0EBEC07F0270E0C6E02C10BF018
:1030C000EBEC07F0280E0C6E03C10BF0EBEC07F0F5
:1030D00000C153F501C154F502C155F503C156F5C0
:1030E00000C157F501C158F502C159F503C15AF5A0
:1030F000EFEF18F004014D0E826FF8EC0AF0290E84
:103100000C6E00C10BF0EBEC07F000C15BF500C1E9
:103110005CF5EFEF18F004014C0E826FF8EC0AF04A
:103120000401540E826FF8EC0AF004012C0E826F39
:10313000F8EC0AF084C32AF185C32BF186C32CF185
:1031400087C32DF188C32EF189C32FF18AC330F1D3
:103150008BC331F18DC332F18EC333F1010108EC21
:1031600027F07FEC26F00101000E046F000E056FC2
:10317000010E066F000E076FD0EC25F0210E0C6ECD
:1031800000C10BF0EBEC07F0220E0C6E01C10BF04E
:10319000EBEC07F0230E0C6E02C10BF0EBEC07F02A
:1031A000240E0C6E03C10BF0EBEC07F000C15DF5D3
:1031B00001C15EF502C15FF503C160F5EFEF18F0E4
:1031C00004014C0E826FF8EC0AF00401490E826F84
:1031D000F8EC0AF004012C0E826FF8EC0AF0250ED0
:1031E00002EC08F0E8CF00F1260E02EC08F0E8CF80
:1031F00001F1270E02EC08F0E8CF02F1280E02ECF4
:1032000008F0E8CF03F15DEC26F040EC24F0040177
:10321000730E826FF8EC0AF004012C0E826FF8EC4A
:103220000AF0BAEC26F0290E02EC08F0E8CF00F123
:103230005DEC26F040EC24F00401730E826FF8EC94
:103240000AF004012C0E826FF8EC0AF057C500F169
:1032500058C501F159C502F15AC503F15DEC26F0DC
:1032600040EC24F00401730E826FF8EC0AF00401C4
:103270002C0E826FF8EC0AF0BAEC26F05CC500F177
:103280005DEC26F040EC24F004016D0E826FF8EC4A
:103290000AF004012C0E826FF8EC0AF05DC500F113
:1032A0005EC501F15FC502F160C503F114EC20F0C9
:1032B00004012C0E826FF8EC0AF002EC0BF0F9EF2F
:1032C0001FF083C32AF184C32BF185C32CF186C37D
:1032D0002DF187C32EF188C32FF189C330F18AC342
:1032E00031F18BC332F18CC333F1010108EC27F0CB
:1032F0007FEC26F0160E0C6E00C10BF0EBEC07F025
:10330000170E0C6E01C10BF0EBEC07F0180E0C6EF3
:1033100002C10BF0EBEC07F0190E0C6E03C10BF0C1
:10332000EBEC07F000C18AF101C18BF102C18CF115
:1033300003C18DF100C18EF101C18FF102C190F185
:1033400003C191F143EF1AF083C32AF184C32BF137
:1033500085C32CF186C32DF187C32EF188C32FF1CD
:1033600089C330F18AC331F18BC332F18CC333F19D
:10337000010108EC27F07FEC26F000C18AF101C1C1
:103380008BF102C18CF103C18DF100C18EF101C13D
:103390008FF102C190F103C191F143EF1AF083C3A1
:1033A0002AF184C32BF185C32CF186C32DF187C389
:1033B0002EF188C32FF189C330F18AC331F18CC358
:1033C00032F18DC333F1010108EC27F07FEC26F0D8
:1033D0000101000E046F000E056F010E066F000E56
:1033E000076FD0EC25F01A0E0C6E00C10BF0EBEC61
:1033F00007F01B0E0C6E01C10BF0EBEC07F01C0E7E
:103400000C6E02C10BF0EBEC07F01D0E0C6E03C14D
:103410000BF0EBEC07F000C192F101C193F102C196
:1034200094F103C195F143EF1AF083C32AF184C3E9
:103430002BF185C32CF186C32DF187C32EF188C3F0
:103440002FF189C330F18AC331F18CC332F18DC3BE
:1034500033F1010108EC27F07FEC26F00101000EAA
:10346000046F000E056F010E066F000E076FD0ECA3
:1034700025F000C192F101C193F102C194F103C1A1
:1034800095F143EF1AF0160E02EC08F0E8CF00F1C8
:10349000170E02EC08F0E8CF01F1180E02EC08F06C
:1034A000E8CF02F1190E02EC08F0E8CF03F15DEC71
:1034B00026F040EC24F00401730E826FF8EC0AF061
:1034C00004012C0E826FF8EC0AF08AC100F18BC166
:1034D00001F18CC102F18DC103F15DEC26F040ECED
:1034E00024F00401730E826FF8EC0AF004012C0E34
:1034F000826FF8EC0AF01A0E02EC08F0E8CF00F147
:103500001B0E02EC08F0E8CF01F11C0E02EC08F0F3
:10351000E8CF02F11D0E02EC08F0E8CF03F114EC45
:1035200020F004012C0E826FF8EC0AF092C100F139
:1035300093C101F194C102F195C103F114EC20F0A3
:1035400002EC0BF0F9EF1FF00401690E826FF8EC4A
:103550000AF004012C0E826FF8EC0AF00101040E4F
:10356000006F000E016F000E026F000E036F5DEC26
:1035700026F02CC182F40401300E8227F8EC0AF008
:103580002DC182F40401300E8227F8EC0AF02EC11E
:1035900082F40401300E8227F8EC0AF02FC182F485
:1035A0000401300E8227F8EC0AF030C182F40401E5
:1035B000300E8227F8EC0AF031C182F40401300E9B
:1035C0008227F8EC0AF032C182F40401300E82271F
:1035D000F8EC0AF033C182F40401300E8227F8ECD3
:1035E0000AF004012C0E826FF8EC0AF001010B0EB8
:1035F000006F000E016F000E026F000E036F5DEC96
:1036000026F02CC182F40401300E8227F8EC0AF077
:103610002DC182F40401300E8227F8EC0AF02EC18D
:1036200082F40401300E8227F8EC0AF02FC182F4F4
:103630000401300E8227F8EC0AF030C182F4040154
:10364000300E8227F8EC0AF031C182F40401300E0A
:103650008227F8EC0AF032C182F40401300E82278E
:10366000F8EC0AF033C182F40401300E8227F8EC42
:103670000AF004012C0E826FF8EC0AF001011D0E15
:10368000006F000E016F000E026F000E036F5DEC05
:1036900026F02CC182F40401300E8227F8EC0AF0E7
:1036A0002DC182F40401300E8227F8EC0AF02EC1FD
:1036B00082F40401300E8227F8EC0AF02FC182F464
:1036C0000401300E8227F8EC0AF030C182F40401C4
:1036D000300E8227F8EC0AF031C182F40401300E7A
:1036E0008227F8EC0AF032C182F40401300E8227FE
:1036F000F8EC0AF033C182F40401300E8227F8ECB2
:103700000AF004012C0E826FF8EC0AF0200EF86E1D
:10371000F76AF66A04010900F5CF82F4F8EC0AF0C2
:103720000900F5CF82F4F8EC0AF00900F5CF82F435
:10373000F8EC0AF00900F5CF82F4F8EC0AF0090081
:10374000F5CF82F4F8EC0AF00900F5CF82F4F8EC3A
:103750000AF00900F5CF82F4F8EC0AF00900F5CF81
:1037600082F4F8EC0AF002EC0BF0F9EF1FF0835151
:10377000630AD8A4F9EF1FF08451610AD8A4F9EFC5
:103780001FF085516C0AD8A4F9EF1FF08651410A49
:1037900042E08651440A1BE08651420AD8B41EEF2B
:1037A0001CF08651350AD8B483EF21F08651360AD1
:1037B000D8B4D8EF21F08651370AD8B441EF22F0BF
:1037C0008651380AD8B49FEF22F0F9EF1FF007981E
:1037D000079A04017A0E826FF8EC0AF00401780E61
:1037E000826FF8EC0AF00401640E826FF8EC0AF0C4
:1037F00081A802EF1CF00401550E826FF8EC0AF06C
:1038000007EF1CF004014C0E826FF8EC0AF002EC9A
:103810000BF0F9EF1FF00788079A04017A0E826F08
:10382000F8EC0AF00401410E826FF8EC0AF0040192
:10383000610E826FF8EC0AF0F8EF1BF00798078A28
:1038400004017A0E826FF8EC0AF00401420E826FD6
:10385000F8EC0AF00401610E826FF8EC0AF0F8EF60
:103860001BF0010166673CEF1CF067673CEF1CF042
:1038700068673CEF1CF0696754EF1CF04F6748EF36
:103880001CF0506748EF1CF0516748EF1CF052677E
:1038900054EF1CF00101000E006F000E016F000ECE
:1038A000026F000E036F12000101620E046F010E21
:1038B000056F000E066F000E076F66C100F167C14D
:1038C00001F168C102F169C103F1BFEC25F003BF4A
:1038D000D8EF1CF00101000E046FA80E056F550E05
:1038E000066F020E076F66C100F167C101F168C182
:1038F00002F169C103F166C186F167C187F168C150
:1039000088F169C189F1BFEC25F003BF91EF1CF08C
:103910000101000E866FA80E876F550E886F020E8C
:10392000896F0E0E02EC08F0E8CF18F10F0E02ECD2
:1039300008F0E8CF19F1100E02EC08F0E8CF1AF108
:10394000110E02EC08F0E8CF1BF108EC25F086C15F
:1039500004F187C105F188C106F189C107F1BFEC07
:1039600025F00782CCEC24F008EC25F00792CCEC93
:1039700024F086C100F187C101F188C102F189C13B
:1039800003F10792CCEC24F0CC0E046FE00E056F2F
:10399000870E066F050E076FBFEC25F000C118F10A
:1039A00001C119F102C11AF103C11BF110EF1DF0A1
:1039B0000101800E006F1A0E016F060E026F000EDD
:1039C000036F4FC104F150C105F151C106F152C15D
:1039D00007F1BFEC25F003AFF1EF1CF0BAEC26F0D5
:1039E00012000E0E02EC08F0E8CF18F10F0E02ECF8
:1039F00008F0E8CF19F1100E02EC08F0E8CF1AF148
:103A0000110E02EC08F0E8CF1BF14FC100F150C1DC
:103A100001F151C102F152C103F10782CCEC24F053
:103A200018C100F119C101F11AC102F11BC103F162
:103A300012000401730E826FF8EC0AF004012C0EE0
:103A4000826FF8EC0AF0078462C166F163C167F126
:103A500064C168F165C169F14BC14FF14CC150F1CE
:103A60004DC151F14EC152F157C159F158C15AF1EE
:103A700007943FEC1DF002EC0BF0F9EF1FF066C16C
:103A800000F167C101F168C102F169C103F10101EF
:103A90005DEC26F040EC24F00401630E826FF8EC3C
:103AA0000AF004012C0E826FF8EC0AF04FC100F10D
:103AB00050C101F151C102F152C103F101015DECAC
:103AC00026F040EC24F00401660E826FF8EC0AF058
:103AD00004012C0E826FF8EC0AF0BAEC26F059C102
:103AE00000F15AC101F101015DEC26F040EC24F037
:103AF0000401740E826FF8EC0AF0120010820401C7
:103B0000530E826FF8EC0AF004012C0E826FF8EC71
:103B10000AF083C32AF184C32BF185C32CF186C339
:103B20002DF187C32EF188C32FF189C330F18AC3E9
:103B300031F18BC332F18CC333F1010108EC27F072
:103B40007FEC26F000C166F101C167F102C168F1A6
:103B500003C169F18EC32AF18FC32BF190C32CF1FD
:103B600091C32DF192C32EF193C32FF194C330F181
:103B700095C331F196C332F197C333F1010108ECDB
:103B800027F07FEC26F000C14FF101C150F102C1D6
:103B900051F103C152F1FBEC26F099C32FF19AC306
:103BA00030F19BC331F19CC332F19DC333F101016C
:103BB00008EC27F07FEC26F000C159F101C15AF161
:103BC0003FEC1DF004012C0E826FF8EC0AF0F0EFD0
:103BD0001DF08251520A03E10F82F0EF1DF00F92A7
:103BE0008251750A03E11084F7EF1DF010948251A1
:103BF000550A03E11086FEEF1DF01096078410B2FF
:103C00005BEF1EF010A447EF1EF0B6C166F1B7C11E
:103C100067F1B8C168F1B9C169F1BAC16AF1BBC154
:103C20006BF1BCC16CF1BDC16DF1BEC16EF1BFC124
:103C30006FF1C0C170F1C1C171F1C2C172F1C3C1F4
:103C400073F1C4C174F1C5C175F1C6C176F1C7C1C4
:103C500077F1C8C178F1C9C179F1CAC17AF1CBC194
:103C60007BF1CCC17CF1CDC17DF1CEC17EF1CFC164
:103C70007FF1D0C180F1D1C181F1D2C182F1D3C134
:103C800083F1D4C184F1D5C185F14FEF1EF062C13B
:103C900066F163C167F164C168F165C169F14BC147
:103CA0004FF14CC150F14DC151F14EC152F157C1CC
:103CB00059F158C15AF107940FA07DEF1EF0010190
:103CC00092676AEF1EF093676AEF1EF094676AEFDF
:103CD0001EF095676EEF1EF07DEF1EF031EC1CF0CC
:103CE00092C104F193C105F194C106F195C107F1A8
:103CF000BFEC25F003BFC1EF1FF031EC1CF0010158
:103D0000000E046F000E056F010E066F000E076FA8
:103D1000F0EC25F010A494EF1EF00401750E826FF4
:103D2000F8EC0AF099EF1EF00401720E826FF8ECC5
:103D30000AF004012C0E826FF8EC0AF05DEC26F01C
:103D40002967A8EF1EF00401200E826FABEF1EF072
:103D500004012D0E826FF8EC0AF030C182F40401E8
:103D6000300E8227F8EC0AF031C182F40401300EE3
:103D70008227F8EC0AF004012E0E826FF8EC0AF0AC
:103D800032C182F40401300E8227F8EC0AF033C10C
:103D900082F40401300E8227F8EC0AF004016D0E63
:103DA000826FF8EC0AF004012C0E826FF8EC0AF036
:103DB0004FC100F150C101F151C102F152C103F1F3
:103DC00001015DEC26F040EC24F00401480E826F06
:103DD000F8EC0AF004017A0E826FF8EC0AF00401A4
:103DE0002C0E826FF8EC0AF066C100F167C101F198
:103DF00068C102F169C103F101015DEC26F040ECFC
:103E000024F00401630E826FF8EC0AF004012C0E1A
:103E1000826FF8EC0AF066C100F167C101F168C178
:103E200002F169C103F101010A0E046F000E056F72
:103E3000000E066F000E076FD0EC25F0000E046F29
:103E4000120E056F000E066F000E076FF0EC25F0E6
:103E50005DEC26F02AC182F40401300E8227F8ECD2
:103E60000AF02BC182F40401300E8227F8EC0AF02C
:103E70002CC182F40401300E8227F8EC0AF02DC127
:103E800082F40401300E8227F8EC0AF02EC182F48D
:103E90000401300E8227F8EC0AF02FC182F40401ED
:103EA000300E8227F8EC0AF030C182F40401300EA3
:103EB0008227F8EC0AF004012E0E826FF8EC0AF06B
:103EC00031C182F40401300E8227F8EC0AF032C1CD
:103ED00082F40401300E8227F8EC0AF033C182F438
:103EE0000401300E8227F8EC0AF00401730E826F91
:103EF000F8EC0AF004012C0E826FF8EC0AF0BAEC30
:103F000026F059C100F15AC101F123EC21F00FB2A2
:103F10008DEF1FF00FA0BFEF1FF004012C0E826F7A
:103F2000F8EC0AF0200EF86EF76AF66A0401090050
:103F3000F5CF82F4F8EC0AF00900F5CF82F4F8EC42
:103F40000AF00900F5CF82F4F8EC0AF00900F5CF89
:103F500082F4F8EC0AF00900F5CF82F4F8EC0AF0EC
:103F60000900F5CF82F4F8EC0AF00900F5CF82F4ED
:103F7000F8EC0AF00900F5CF82F4F8EC0AF002EC54
:103F80000BF00F90F9EF1FF00401630E826FF8EC55
:103F90000AF004012C0E826FF8EC0AF0FFEC1FF01F
:103FA00004012C0E826FF8EC0AF072EC20F0040190
:103FB0002C0E826FF8EC0AF0EEEC20F004012C0ECF
:103FC000826FF8EC0AF00101F80E006FCD0E016F60
:103FD000660E026F030E036F14EC20F004012C0E2A
:103FE000826FF8EC0AF004EC21F002EC0BF0F9EF30
:103FF0001FF00301C26B0790109208EF23F0D890D6
:104000000E0E02EC08F0E8CF00F10F0E02EC08F003
:10401000E8CF01F1100E02EC08F0E8CF02F1110E2A
:1040200002EC08F0E8CF03F10101000E046F000E6E
:10403000056F010E066F000E076FF0EC25F05DECCA
:1040400026F02AC182F40401300E8227F8EC0AF02F
:104050002BC182F40401300E8227F8EC0AF02CC147
:1040600082F40401300E8227F8EC0AF02DC182F4AC
:104070000401300E8227F8EC0AF02EC182F404010C
:10408000300E8227F8EC0AF02FC182F40401300EC2
:104090008227F8EC0AF030C182F40401300E822746
:1040A000F8EC0AF031C182F40401300E8227F8ECFA
:1040B0000AF004012E0E826FF8EC0AF032C182F48D
:1040C0000401300E8227F8EC0AF033C182F40401B7
:1040D000300E8227F8EC0AF004016D0E826FF8ECC6
:1040E0000AF01200120E02EC08F0E8CF00F1130EF5
:1040F00002EC08F0E8CF01F1140E02EC08F0E8CF72
:1041000002F1150E02EC08F0E8CF03F101010A0EEE
:10411000046F000E056F000E066F000E076FD0ECE7
:1041200025F0000E046F120E056F000E066F000ED4
:10413000076FF0EC25F05DEC26F02AC182F4040153
:10414000300E8227F8EC0AF02BC182F40401300E05
:104150008227F8EC0AF02CC182F40401300E822789
:10416000F8EC0AF02DC182F40401300E8227F8EC3D
:104170000AF02EC182F40401300E8227F8EC0AF016
:104180002FC182F40401300E8227F8EC0AF030C10E
:1041900082F40401300E8227F8EC0AF004012E0E9E
:1041A000826FF8EC0AF031C182F40401300E8227EC
:1041B000F8EC0AF032C182F40401300E8227F8ECE8
:1041C0000AF033C182F40401300E8227F8EC0AF0C1
:1041D0000401730E826FF8EC0AF012000A0E02EC72
:1041E00008F0E8CF00F10B0E02EC08F0E8CF01F187
:1041F0000C0E02EC08F0E8CF02F10D0E02EC08F014
:10420000E8CF03F123EF21F0060E02EC08F0E8CF2F
:1042100000F1070E02EC08F0E8CF01F1080E02EC05
:1042200008F0E8CF02F1090E02EC08F0E8CF03F144
:1042300023EF21F00101BAEC26F0078457C100F109
:1042400058C101F107940101E80E046F800E056F5B
:10425000000E066F000E076FD0EC25F0000E046F05
:10426000040E056F000E066F000E076FF0EC25F0D0
:10427000880E046F130E056F000E066F000E076F99
:10428000BFEC25F00A0E046F000E056F000E066FDE
:10429000000E076FF0EC25F05DEC26F001012967B8
:1042A00057EF21F00401200E826F5AEF21F0040134
:1042B0002D0E826FF8EC0AF030C182F40401300E4A
:1042C0008227F8EC0AF031C182F40401300E822713
:1042D000F8EC0AF032C182F40401300E8227F8ECC7
:1042E0000AF004012E0E826FF8EC0AF033C182F45A
:1042F0000401300E8227F8EC0AF00401430E826FAD
:10430000F8EC0AF0120087C32AF188C32BF189C3A5
:104310002CF18AC32DF18BC32EF18CC32FF18DC3E9
:1043200030F18EC331F190C332F191C333F1010109
:10433000296B08EC27F07FEC26F00101000E046FDA
:10434000000E056F010E066F000E076FD0EC25F012
:104350000E0E0C6E00C10BF0EBEC07F00F0E0C6EA6
:1043600001C10BF0EBEC07F0100E0C6E02C10BF06C
:10437000EBEC07F0110E0C6E03C10BF0EBEC07F049
:1043800004017A0E826FF8EC0AF004012C0E826FA1
:10439000F8EC0AF00401350E826FF8EC0AF0040123
:1043A0002C0E826FF8EC0AF0FFEC1FF007EF1CF008
:1043B00087C32AF188C32BF189C32CF18AC32DF15D
:1043C0008BC32EF18CC32FF18DC330F18EC331F12D
:1043D00090C332F191C333F10101296B08EC27F04E
:1043E0007FEC26F0880E046F130E056F000E066F2B
:1043F000000E076FC4EC25F0000E046F040E056F6D
:10440000000E066F000E076FD0EC25F00101E80EDC
:10441000046F800E056F000E066F000E076FF0EC44
:1044200025F00A0E0C6E00C10BF0EBEC07F00B0E42
:104430000C6E01C10BF0EBEC07F00C0E0C6E02C120
:104440000BF0EBEC07F00D0E0C6E03C10BF0EBEC78
:1044500007F004017A0E826FF8EC0AF004012C0ECA
:10446000826FF8EC0AF00401360E826FF8EC0AF065
:1044700004012C0E826FF8EC0AF0EEEC20F007EF4E
:104480001CF087C32AF188C32BF189C32CF18AC39E
:104490002DF18BC32EF18CC32FF18DC330F18FC35F
:1044A00031F190C332F191C333F1010108EC27F0EF
:1044B0007FEC26F0000E046F120E056F000E066FE3
:1044C000000E076FD0EC25F001010A0E046F000EFC
:1044D000056F000E066F000E076FF0EC25F0120E50
:1044E0000C6E00C10BF0EBEC07F0130E0C6E01C16B
:1044F0000BF0EBEC07F0140E0C6E02C10BF0EBECC2
:1045000007F0150E0C6E03C10BF0EBEC07F0040185
:104510007A0E826FF8EC0AF004012C0E826FF8EC30
:104520000AF00401370E826FF8EC0AF004012C0E39
:10453000826FF8EC0AF072EC20F007EF1CF087C3F2
:104540002AF188C32BF189C32CF18AC32DF18BC3C7
:104550002EF18CC32FF18DC330F18EC331F190C396
:1045600032F191C333F10101296B08EC27F07FECA4
:1045700026F0880E046F130E056F000E066F000EF6
:10458000076FC4EC25F0000E046F040E056F000EDB
:10459000066F000E076FD0EC25F00101E80E046FE6
:1045A000800E056F000E066F000E076FF0EC25F011
:1045B000060E0C6E00C10BF0EBEC07F0070E0C6E54
:1045C00001C10BF0EBEC07F0080E0C6E02C10BF012
:1045D000EBEC07F0090E0C6E03C10BF0EBEC07F0EF
:1045E00004017A0E826FF8EC0AF004012C0E826F3F
:1045F000F8EC0AF00401380E826FF8EC0AF00401BE
:104600002C0E826FF8EC0AF004EC21F007EF1CF09E
:1046100081A8C6EF23F007A87FEF23F00101800EE9
:10462000006F1A0E016F060E026F000E036F4BC172
:1046300004F14CC105F14DC106F14EC107F1BFECCB
:1046400025F003BFC6EF23F03AEC24F04BC100F194
:104650004CC101F14DC102F14EC103F10782CCEC16
:1046600024F018C104F119C105F11AC106F11BC1EA
:1046700007F1F80E006FCD0E016F660E026F030E8C
:10468000036FBFEC25F00E0E0C6E00C10BF0EBECCF
:1046900007F00F0E0C6E01C10BF0EBEC07F0100EE3
:1046A0000C6E02C10BF0EBEC07F0110E0C6E03C1A7
:1046B0000BF0EBEC07F007840101BAEC26F057C1D0
:1046C00000F158C101F107940A0E0C6E00C10BF005
:1046D000EBEC07F00B0E0C6E01C10BF0EBEC07F0EE
:1046E0000C0E0C6E02C10BF0EBEC07F00D0E0C6E15
:1046F00003C10BF0EBEC07F00798C6EF23F007AA15
:10470000C6EF23F007840101BAEC26F057C100F18F
:1047100058C101F10794060E0C6E00C10BF0EBECD2
:1047200007F0070E0C6E01C10BF0EBEC07F0080E62
:104730000C6E02C10BF0EBEC07F0090E0C6E03C11E
:104740000BF0EBEC07F0078462C100F163C101F1EB
:1047500064C102F165C103F10794120E0C6E00C131
:104760000BF0EBEC07F0130E0C6E01C10BF0EBEC51
:1047700007F0140E0C6E02C10BF0EBEC07F0150EF7
:104780000C6E03C10BF0EBEC07F0079A04018051AB
:1047900081197F0B0BE09EA809D014EE00F0815127
:1047A0007F0BE126E750812B0F01AD6E05012F51E4
:1047B000010A13E081AAEDEF23F005012F51000A51
:1047C0000AE00FB8EDEF23F005013067EDEF23F0BD
:1047D0000FB8EDEF23F0B8EF30F081B802EF24F01E
:1047E00023EC29F005012F51020A02E002EF24F028
:1047F0005C2F02EF24F05BC55CF50501010E306F04
:104800003C0E316F61EF0AF018C100F119C101F1DE
:104810001AC102F11BC103F1000E046F000E056FF7
:10482000010E066F000E076FF0EC25F029A12FEFA7
:1048300024F02051D8B42FEF24F018C100F119C191
:1048400001F11AC102F11BC103F1000E046F000E49
:10485000056F0A0E066F000E076FF0EC25F01200D0
:1048600001010451001305510113065102130751B0
:10487000031312000101186B196B1A6B1B6B1200EA
:104880002AC182F40401300E8227F8EC0AF02BC111
:1048900082F40401300E8227F8EC0AF02CC182F475
:1048A0000401300E8227F8EC0AF02DC182F40401D5
:1048B000300E8227F8EC0AF02EC182F40401300E8B
:1048C0008227F8EC0AF02FC182F40401300E82270F
:1048D000F8EC0AF030C182F40401300E8227F8ECC3
:1048E0000AF031C182F40401300E8227F8EC0AF09C
:1048F00032C182F40401300E8227F8EC0AF033C191
:1049000082F40401300E8227F8EC0AF012002FC165
:1049100082F40401300E8227F8EC0AF030C182F4F0
:104920000401300E8227F8EC0AF031C182F4040150
:10493000300E8227F8EC0AF032C182F40401300E06
:104940008227F8EC0AF033C182F40401300E82278A
:10495000F8EC0AF01200060E116E060E126E060E2C
:10496000136E112EB1EF24F0122EB1EF24F0132E9E
:10497000B1EF24F08B84020E116E020E126E020E45
:10498000136E112EC1EF24F0122EC1EF24F0132E5E
:10499000C1EF24F08B9412000101005305E1015393
:1049A00003E1025301E1002B8FEC25F0BAEC26F075
:1049B0003951006F3A51016F420E046F4B0E056F73
:1049C000000E066F000E076FD0EC25F000C104F159
:1049D00001C105F102C106F103C107F118C100F1DF
:1049E00019C101F11AC102F11BC103F107B2FDEFB8
:1049F00024F0C4EC25F0FFEF24F0BFEC25F000C15B
:104A000018F101C119F102C11AF103C11BF1120021
:104A1000BAEC26F059C100F15AC101F1060E02ECC0
:104A200008F0E8CF04F1070E02EC08F0E8CF05F13A
:104A3000080E02EC08F0E8CF06F1090E02EC08F0CF
:104A4000E8CF07F1BFEC25F000C124F101C125F149
:104A500002C126F103C127F1290E046F000E056F74
:104A6000000E066F000E076FD0EC25F0EE0E046FFF
:104A7000430E056F000E066F000E076FC4EC25F0A5
:104A800024C104F125C105F126C106F127C107F1B2
:104A9000D0EC25F000C11CF101C11DF102C11EF1D5
:104AA00003C11FF1120E02EC08F0E8CF04F1130E5F
:104AB00002EC08F0E8CF05F1140E02EC08F0E8CFA4
:104AC00006F1150E02EC08F0E8CF07F10D0E006FAD
:104AD000000E016F000E026F000E036FD0EC25F088
:104AE000180E046F000E056F000E066F000E076FA4
:104AF000F0EC25F01CC104F11DC105F11EC106F149
:104B00001FC107F1C4EC25F06A0E046F2A0E056F71
:104B1000000E066F000E076FBFEC25F01200BF0EEF
:104B2000FA6E200E3A6F396BD89000370137023792
:104B30000337D8B0A0EF25F03A2F95EF25F03907CD
:104B40003A070353D8B412000331070B80093F6FB3
:104B500003390F0B010F396F80EC5FF0406F39059F
:104B600080EC5FF0405D405F396B3F33D8B0392750
:104B700039333FA9B5EF25F0405139271200010123
:104B8000DFEC26F0D8B01200010103510719346F91
:104B9000A2EC26F0D8900751031934AF800F120011
:104BA0000101346BC6EC26F0D8A0DCEC26F0D8B0BE
:104BB0001200B1EC26F0BAEC26F01F0E366FF2ECC4
:104BC00026F00B35D8B0A2EC26F0D8A00335D8B02B
:104BD0001200362FDFEF25F034B1C9EC26F01200B9
:104BE0000101346B04510511061107110008D8A00A
:104BF000C6EC26F0D8A0DCEC26F0D8B01200086B8A
:104C0000096B0A6B0B6BF2EC26F01F0E366FF2ECA1
:104C100026F007510B5DD8A41AEF26F006510A5D65
:104C2000D8A41AEF26F00551095DD8A41AEF26F092
:104C30000451085DD8A02DEF26F00451085F0551FE
:104C4000D8A0053D095F0651D8A0063D0A5F07516F
:104C5000D8A0073D0B5FD8900081362F07EF26F0D4
:104C600034B1C9EC26F0346BC6EC26F0D890F6ECE3
:104C700026F007510B5DD8A44AEF26F006510A5DD5
:104C8000D8A44AEF26F00551095DD8A44AEF26F0D2
:104C90000451085DD8A059EF26F0003F59EF26F0E7
:104CA000013F59EF26F0023F59EF26F0032BD8B40D
:104CB000120034B1C9EC26F012000101346BC6ECCD
:104CC00026F0D8B01200FBEC26F0200E366F00372D
:104CD00001370237033711EE33F00A0E376FE7362C
:104CE0000A0EE75CD8B0E76EE552372F6FEF26F07B
:104CF000362F67EF26F034B12981D89012000101D8
:104D00000A0E346F200E366F11EE29F03451376FD2
:104D10000A0ED890E652D8B0E726E732372F8AEF4E
:104D200026F00333023301330033362F84EF26F0AD
:104D3000E750FF0FD8A00335D8B0120029B1C9EC55
:104D400026F01200045100270551D8B0053D012777
:104D50000651D8B0063D02270751D8B0073D0327BA
:104D600012000051086F0151096F02510A6F03517F
:104D70000B6F12000101006B016B026B036B1200E1
:104D80000101046B056B066B076B12000335D8A09D
:104D900012000351800B001F011F021F031F003F61
:104DA000D9EF26F0013FD9EF26F0023FD9EF26F0E8
:104DB000032B342B032512000735D8A0120007510E
:104DC000800B041F051F061F071F043FEFEF26F08F
:104DD000053FEFEF26F0063FEFEF26F0072B342BD1
:104DE0000725120000370137023703370837093724
:104DF0000A370B3712000101296B2A6B2B6B2C6BC6
:104E00002D6B2E6B2F6B306B316B326B336B120053
:104E100001012A510F0B2A6F2B510F0B2B6F2C51B5
:104E20000F0B2C6F2D510F0B2D6F2E510F0B2E6F63
:104E30002F510F0B2F6F30510F0B306F31510F0B64
:104E4000316F32510F0B326F33510F0B336F120032
:104E5000899C000EC76E200EC66E9E96C69EC50E1D
:104E6000C96EFF0E9EB602D0E82EFCD79E96C69E57
:104E7000000EC96EFF0E9EB602D0E82EFCD7C9CF39
:104E800000F69E96C69E000EC96EFF0E9EB602D01C
:104E9000E82EFCD7C9CF01F6898C1200000EC76E30
:104EA000200EC66E899C9E96C69EC80EC96EFF0EC9
:104EB0009EB602D0E82EFCD79E96C69E000EC96E06
:104EC000FF0E9EB602D0E82EFCD7C9CF02F69E9602
:104ED000C69E000EC96EFF0E9EB602D0E82EFCD70D
:104EE000C9CF03F6898C899C9E96C69ECA0EC96E50
:104EF000FF0E9EB602D0E82EFCD79E96C69E000EF0
:104F0000C96EFF0E9EB602D0E82EFCD7C9CF0AF6B6
:104F10009E96C69E000EC96EFF0E9EB602D0E82E6B
:104F2000FCD7C9CF0BF6898C899C9E96C69ECC0E69
:104F3000C96EFF0E9EB602D0E82EFCD79E96C69E86
:104F4000000EC96EFF0E9EB602D0E82EFCD7C9CF68
:104F500012F69E96C69E000EC96EFF0E9EB602D039
:104F6000E82EFCD7C9CF13F6898C1200000EC76E4D
:104F7000200EC66E899C9E96C69EE80EC96EFF0ED8
:104F80009EB602D0E82EFCD79E96C69E000EC96E35
:104F9000FF0E9EB602D0E82EFCD7C9CF1AF69E9619
:104FA000C69E000EC96EFF0E9EB602D0E82EFCD73C
:104FB000C9CF1BF6898C899C9E96C69EEA0EC96E47
:104FC000FF0E9EB602D0E82EFCD79E96C69E000E1F
:104FD000C96EFF0E9EB602D0E82EFCD7C9CF22F6CE
:104FE0009E96C69E000EC96EFF0E9EB602D0E82E9B
:104FF000FCD7C9CF23F6898C899C9E96C69EEC0E61
:10500000C96EFF0E9EB602D0E82EFCD79E96C69EB5
:10501000000EC96EFF0E9EB602D0E82EFCD7C9CF97
:105020002AF69E96C69E000EC96EFF0E9EB602D050
:10503000E82EFCD7C9CF2BF6898C1200000EC76E64
:10504000200EC66E899C9E96C69E240EC96EFF0ECB
:105050009EB602D0E82EFCD79E96C69EE40EC96E80
:10506000FF0E9EB602D0E82EFCD7898C899C9E96B6
:10507000C69E200EC96EFF0E9EB602D0E82EFCD74B
:105080009E96C69E5F0EC96EFF0E9EB602D0E82E9B
:10509000FCD7898C899C9E96C69E210EC96EFF0EF8
:1050A0009EB602D0E82EFCD79E96C69EC00EC96E54
:1050B000FF0E9EB602D0E82EFCD7898C899C9E9666
:1050C000C69E260EC96EFF0E9EB602D0E82EFCD7F5
:1050D0009E96C69E000EC96EFF0E9EB602D0E82EAA
:1050E000FCD7898C12008984000EC76E220EC66E12
:1050F0009E96C69E000EC96EFF0E9EB602D0E82E8A
:10510000FCD79E96C69E000EC96EFF0E9EB602D0BC
:10511000E82EFCD7C9CFABF59E96C69E000EC96E91
:10512000FF0E9EB602D0E82EFCD7C9CFACF59E96F6
:10513000C69E000EC96EFF0E9EB602D0E82EFCD7AA
:10514000C9CFADF59E96C69E000EC96EFF0E9EB6E7
:1051500002D0E82EFCD7C9CFAEF59E96C69E000EB3
:10516000C96EFF0E9EB602D0E82EFCD7C9CFAFF5B0
:105170009E96C69E000EC96EFF0E9EB602D0E82E09
:10518000FCD7C9CFB0F59E96C69E000EC96EFF0E25
:105190009EB602D0E82EFCD7C9CFB1F5899426EC93
:1051A0002BF012008984000EC76E220EC66E9E96EA
:1051B000C69E800EC96EFF0E9EB602D0E82EFCD7AA
:1051C0009E96C69EABC5C9FFFF0E9EB602D0E82EC6
:1051D000FCD79E96C69EACC5C9FFFF0E9EB602D0F8
:1051E000E82EFCD79E96C69EADC5C9FFFF0E9EB6A3
:1051F00002D0E82EFCD79E96C69EAEC5C9FFFF0E14
:105200009EB602D0E82EFCD79E96C69EAFC5C9FFBB
:10521000FF0E9EB602D0E82EFCD79E96C69EB0C565
:10522000C9FFFF0E9EB602D0E82EFCD79E96C69E02
:10523000B1C5C9FFFF0E9EB602D0E82EFCD78994F7
:1052400026EC2BF012008984000EC76E220EC66E6B
:105250009E96C69E070EC96EFF0E9EB602D0E82E21
:10526000FCD79E96C69E000EC96EFF0E9EB602D05B
:10527000E82EFCD7C9CFABF59E96C69E000EC96E30
:10528000FF0E9EB602D0E82EFCD7C9CFACF59E9695
:10529000C69E000EC96EFF0E9EB602D0E82EFCD749
:1052A000C9CFADF59E96C69E000EC96EFF0E9EB686
:1052B00002D0E82EFCD7C9CFAEF5899426EC2BF0AE
:1052C0008984000EC76E220EC66E9E96C69E0F0E75
:1052D000C96EFF0E9EB602D0E82EFCD79E96C69EE3
:1052E000000EC96EFF0E9EB602D0E82EFCD7C9CFC5
:1052F000B3F5899426EC2BF012008984000EC76E5A
:10530000220EC66E9E96C69E870EC96EFF0E9EB674
:1053100002D0E82EFCD79E96C69EABC5C9FFFF0EF5
:105320009EB602D0E82EFCD79E96C69EACC5C9FF9D
:10533000FF0E9EB602D0E82EFCD79E96C69EADC547
:10534000C9FFFF0E9EB602D0E82EFCD79E96C69EE1
:10535000AEC5C9FFFF0E9EB602D0E82EFCD78994D9
:1053600026EC2BF089849E96C69E8F0EC96EFF0E8A
:105370009EB602D0E82EFCD79E96C69EB3C5C9FF46
:10538000FF0E9EB602D0E82EFCD7899426EC2BF0B7
:1053900012008984000EC76E220EC66E9E96C69EAF
:1053A000870EC96EFF0E9EB602D0E82EFCD79E96E1
:1053B000C69E000EC96EFF0E9EB602D0E82EFCD728
:1053C0009E96C69E800EC96EFF0E9EB602D0E82E37
:1053D000FCD79E96C69E800EC96EFF0E9EB602D06A
:1053E000E82EFCD79E96C69E800EC96EFF0E9EB616
:1053F00002D0E82EFCD7899426EC2BF089849E9667
:10540000C69E8F0EC96EFF0E9EB602D0E82EFCD748
:105410009E96C69E010EC96EFF0E9EB602D0E82E65
:10542000FCD7899426EC2BF012008984000EC76EFD
:10543000220EC66E9E96C69E870EC96EFF0E9EB643
:1054400002D0E82EFCD79E96C69E000EC96EFF0EB7
:105450009EB602D0E82EFCD79E96C69E000EC96E60
:10546000FF0E9EB602D0E82EFCD79E96C69E800EFA
:10547000C96EFF0E9EB602D0E82EFCD79E96C69E41
:10548000800EC96EFF0E9EB602D0E82EFCD789941E
:1054900026EC2BF089849E96C69E8F0EC96EFF0E59
:1054A0009EB602D0E82EFCD79E96C69E010EC96E0F
:1054B000FF0E9EB602D0E82EFCD7899426EC2BF086
:1054C00012008984000EC76E220EC66E9E96C69E7E
:1054D0008F0EC96EFF0E9EB602D0E82EFCD726ECCA
:1054E0002BF09E96C69E810EC96EFF0E9EB602D010
:1054F000E82EFCD7899426EC2BF08984000EC76E29
:10550000220EC66E9E96C69E8F0EC96EFF0E9EB66A
:1055100002D0E82EFCD726EC2BF09E96C69E010EFC
:10552000C96EFF0E9EB602D0E82EFCD7899426ECF9
:105530002BF089849E96C69E910EC96EFF0E9EB674
:1055400002D0E82EFCD726EC2BF09E96C69EA50E28
:10555000C96EFF0E9EB602D0E82EFCD7899426ECC9
:105560002BF012008984000EC76E220EC66E9E9626
:10557000C69E8F0EC96EFF0E9EB602D0E82EFCD7D7
:1055800026EC2BF09E96C69E810EC96EFF0E9EB62F
:1055900002D0E82EFCD7899426EC2BF012008984E7
:1055A000000EC76E220EC66E9E96C69E8F0EC96EE8
:1055B000FF0E9EB602D0E82EFCD726EC2BF09E966E
:1055C000C69E010EC96EFF0E9EB602D0E82EFCD715
:1055D000899426EC2BF012008984000EC76E220EEF
:1055E000C66E9E96C69E910EC96EFF0E9EB602D0E6
:1055F000E82EFCD726EC2BF09E96C69EA50EC96E13
:10560000FF0E9EB602D0E82EFCD7899426EC2BF034
:1056100012008984000EC76E220EC66E9E96C69E2C
:10562000910EC96EFF0E9EB602D0E82EFCD726EC76
:105630002BF09E96C69E000EC96EFF0E9EB602D03F
:10564000E82EFCD7899426EC2BF01200050EE82EEC
:10565000FED712000501256B266B276B286B899AF4
:10566000400EC76E200EC66E9E96C69E030EC96E75
:10567000FF0E9EB602D0E82EFCD79E96C69E27C58A
:10568000C9FFFF0E9EB602D0E82EFCD79E96C69E9E
:1056900026C5C9FFFF0E9EB602D0E82EFCD79E9607
:1056A000C69E25C5C9FFFF0E9EB602D0E82EFCD7C8
:1056B0009E96C69EC952FF0E9EB602D0E82EFCD71B
:1056C000898A0F01C950FF0A01E1120005012E511C
:1056D000130A05E005012E51170A0CE0120005011E
:1056E000E00E256FFF0E266F0F0E276F000E286F3E
:1056F00083EF2BF00501E00E256FFF0E266FFF0EE6
:10570000276F000E286F899A400EC76E200EC66E56
:105710009E96C69E030EC96EFF0E9EB602D0E82E60
:10572000FCD79E96C69E27C5C9FFFF0E9EB602D027
:10573000E82EFCD79E96C69E26C5C9FFFF0E9EB6D4
:1057400002D0E82EFCD79E96C69E25C5C9FFFF0E47
:105750009EB602D0E82EFCD79E96C69EC952FF0E7A
:105760009EB602D0E82EFCD7898A0F01C950FF0AE5
:105770001DE005012E51130A05E005012E51170AFF
:105780000BE012000501000E256F000E266F100EB3
:10579000276F000E286F12000501000E256F000E06
:1057A000266F000E276F010E286F12000501256B72
:1057B000266B276B286B05012E51130A05E00501A6
:1057C0002E51170A0CE012000501000E216F000E89
:1057D000226F040E236F000E246FF8EF2BF00501EB
:1057E000000E216F000E226F800E236F000E246FBB
:1057F00021C500F122C501F123C502F124C503F141
:1058000025C504F126C505F127C506F128C507F110
:1058100030EC24F000C125F501C126F502C127F5C1
:1058200003C128F5899A400EC76E200EC66E9E965B
:10583000C69E030EC96EFF0E9EB602D0E82EFCD7A0
:105840009E96C69E27C5C9FFFF0E9EB602D0E82EC3
:10585000FCD79E96C69E26C5C9FFFF0E9EB602D0F7
:10586000E82EFCD79E96C69E25C5C9FFFF0E9EB6A4
:1058700002D0E82EFCD79E96C69EC952FF0E9EB659
:1058800002D0E82EFCD7898AC950FF0A08E104C17A
:1058900025F505C126F506C127F507C128F5D890DD
:1058A000050124332333223321332151E00B216FAF
:1058B000216762EF2CF0226762EF2CF0236762EF22
:1058C0002CF02467F8EF2BF00501200E2527E86A5D
:1058D0002623E86A2723E86A28231200E86A0501DC
:1058E0002E51130A06E005012E51170A0BE0020E95
:1058F000120005012851000A03E12751F00B07E0CF
:10590000010E120005012851000A01E0010E1200EB
:1059100029C500F12AC501F12BC502F12CC503F1FF
:1059200025C504F126C505F127C506F128C507F1EF
:10593000BFEC25F003BF12006EEC2CF05FE1899AFA
:10594000400EC76E200EC66E9E96C69E060EC96E8F
:10595000FF0E9EB602D0E82EFCD7898A899A9E96C1
:10596000C69E020EC96EFF0E9EB602D0E82EFCD770
:105970009E96C69E27C5C9FFFF0E9EB602D0E82E92
:10598000FCD79E96C69E26C5C9FFFF0E9EB602D0C6
:10599000E82EFCD79E96C69E25C5C9FFFF0E9EB673
:1059A00002D0E82EFCD79E96C69E000EC96EFF0E52
:1059B0009EB602D0E82EFCD7898A899A9E96C69E0A
:1059C000050EC96EFF0E9EB602D0E82EFCD79E963D
:1059D000C69EC952FF0E9EB602D0E82EFCD7C9B0B3
:1059E000E7EF2CF0898A0501200E2527E86A262397
:1059F000E86A2723E86A282388EF2CF01200899AA6
:105A0000400EC76E200EC66E9E96C69E060EC96ECE
:105A1000FF0E9EB602D0E82EFCD7898A899A9E9600
:105A2000C69EC70EC96EFF0E9EB602D0E82EFCD7EA
:105A3000898A0501256B266B276B286B1200899AD2
:105A4000400EC76E200EC66E9E96C69E050EC96E8F
:105A5000FF0E9EB602D0E82EFCD79E96C69EC95277
:105A6000FF0E9EB602D0E82EFCD7C9CF33F5898A47
:105A70001200899A400EC76E200EC66E9E96C69E74
:105A8000B90EC96EFF0E9EB602D0E82EFCD7898AE9
:105A90001200899A400EC76E200EC66E9E96C69E54
:105AA000AB0EC96EFF0E9EB602D0E82EFCD7898AD7
:105AB000FF0EE82EFED712006EEC2CF0D8A41200D8
:105AC000899A400EC76E200EC66E9E96C69E030E25
:105AD000C96EFF0E9EB602D0E82EFCD79E96C69EDB
:105AE00027C5C9FFFF0E9EB602D0E82EFCD79E96B2
:105AF000C69E26C5C9FFFF0E9EB602D0E82EFCD773
:105B00009E96C69E25C5C9FFFF0E9EB602D0E82E02
:105B1000FCD79E96C69EC952FF0E9EB602D0E82EB6
:105B2000FCD7898A0F01C950FF0AD8A42BEF30F0A7
:105B30000501FE0E336F73EC28F0ABC534F5ACC530
:105B400035F5ADC536F5AEC537F5AFC538F5B0C5D9
:105B500039F5B1C53AF50784B6C166F1B7C167F149
:105B6000B8C168F1B9C169F14BC14FF14CC150F1F5
:105B70004DC151F14EC152F157C159F158C15AF1BD
:105B800031EC1CF000C13BF501C13CF502C13DF513
:105B900003C13EF505015D67D5EF2DF05E67D5EFDA
:105BA0002DF05F67D5EF2DF06067D9EF2DF0E6EFB0
:105BB0002DF05DC504F15EC505F15FC506F160C558
:105BC00007F1BFEC25F003BF2BEF30F059C13FF5D3
:105BD0005AC140F5B5C541F5B6C542F50101036BA3
:105BE000026B1AC600F11BC601F101AFFCEF2DF0EC
:105BF000FF0E026FFF0E036F0101076B066B1CC6E1
:105C000004F11DC605F105AF0AEF2EF0FF0E066F79
:105C1000FF0E076FC4EC25F00101076B066B1EC673
:105C200004F11FC605F105AF1AEF2EF0FF0E066F47
:105C3000FF0E076FC4EC25F00101076B066B20C651
:105C400004F121C605F105AF2AEF2EF0FF0E066F15
:105C5000FF0E076FC4EC25F0D89001010333023327
:105C600001330033D8900101033302330133003391
:105C700000C147F501C148F50101036B026B22C663
:105C800000F123C601F101AF4AEF2EF0FF0E026FC3
:105C9000FF0E036F0101076B066B24C604F125C6D6
:105CA00005F105AF58EF2EF0FF0E066FFF0E076FE0
:105CB000C4EC25F00101076B066B26C604F127C66C
:105CC00005F105AF68EF2EF0FF0E066FFF0E076FB0
:105CD000C4EC25F00101076B066B28C604F129C648
:105CE00005F105AF78EF2EF0FF0E066FFF0E076F80
:105CF000C4EC25F0D89001010333023301330033A3
:105D0000D8900101033302330133003300C149F558
:105D100001C14AF50101036B026B2AC600F12BC6D3
:105D200001F101AF98EF2EF0FF0E026FFF0E036F2F
:105D30000101076B066B2CC604F12DC605F105AFFA
:105D4000A6EF2EF0FF0E066FFF0E076FC4EC25F0D6
:105D50000101076B066B2EC604F12FC605F105AFD6
:105D6000B6EF2EF0FF0E066FFF0E076FC4EC25F0A6
:105D70000101076B066B30C604F131C605F105AFB2
:105D8000C6EF2EF0FF0E066FFF0E076FC4EC25F076
:105D9000D89001010333023301330033D89001015D
:105DA000033302330133003300C14BF501C14CF51D
:105DB0000101036B026B02C600F103C601F101AFE2
:105DC000E6EF2EF0FF0E026FFF0E036F0101076B6F
:105DD000066B04C604F105C605F105AFF4EF2EF01D
:105DE000FF0E066FFF0E076FC4EC25F00101076B75
:105DF000066B06C604F107C605F105AF04EF2FF0E8
:105E0000FF0E066FFF0E076FC4EC25F00101076B54
:105E1000066B08C604F109C605F105AF14EF2FF0B3
:105E2000FF0E066FFF0E076FC4EC25F0D89001013E
:105E30000333023301330033D890010103330233BB
:105E40000133003300C14DF501C14EF50101036B73
:105E5000026B0AC600F10BC601F101AF34EF2FF05F
:105E6000FF0E026FFF0E036F0101076B066B0CC67E
:105E700004F10DC605F105AF42EF2FF0FF0E066FDE
:105E8000FF0E076FC4EC25F00101076B066B0EC611
:105E900004F10FC605F105AF52EF2FF0FF0E066FAC
:105EA000FF0E076FC4EC25F00101076B066B10C6EF
:105EB00004F111C605F105AF62EF2FF0FF0E066F7A
:105EC000FF0E076FC4EC25F0D890010103330233B5
:105ED00001330033D890010103330233013300331F
:105EE00000C14FF501C150F50101036B026B12C6F1
:105EF00000F113C601F101AF82EF2FF0FF0E026F28
:105F0000FF0E036F0101076B066B14C604F115C683
:105F100005F105AF90EF2FF0FF0E066FFF0E076F34
:105F2000C4EC25F00101076B066B16C604F117C619
:105F300005F105AFA0EF2FF0FF0E066FFF0E076F04
:105F4000C4EC25F00101076B066B18C604F119C6F5
:105F500005F105AFB0EF2FF0FF0E066FFF0E076FD4
:105F6000C4EC25F0D8900101033302330133003330
:105F7000D8900101033302330133003300C151F5DE
:105F800001C152F507940501200E326F899A400E27
:105F9000C76E200EC66E9E96C69E060EC96EFF0E7A
:105FA0009EB602D0E82EFCD7898A899A9E96C69E14
:105FB000020EC96EFF0E9EB602D0E82EFCD79E964A
:105FC000C69E27C5C9FFFF0E9EB602D0E82EFCD79D
:105FD0009E96C69E26C5C9FFFF0E9EB602D0E82E2D
:105FE000FCD79E96C69E25C5C9FFFF0E9EB602D061
:105FF000E82EFCD725EE33F0322F02D00BEF30F035
:106000009E96C69EDECFC9FFFF0E9EB602D0E82E3A
:10601000FCD7FCEF2FF0898A899A9E96C69E050EC2
:10602000C96EFF0E9EB602D0E82EFCD79E96C69E85
:10603000C952FF0E9EB602D0E82EFCD7C9B016EFAB
:1060400030F0898A0501200E2527E86A2623E86AB0
:106050002723E86A2823120021C500F122C501F197
:1060600023C502F124C503F1899A400EC76E200EA4
:10607000C66E9E96C69E0B0EC96EFF0E9EB602D0D1
:10608000E82EFCD79E96C69E02C1C9FFFF0E9EB6A3
:1060900002D0E82EFCD79E96C69E01C1C9FFFF0E16
:1060A0009EB602D0E82EFCD79E96C69E00C1C9FFC0
:1060B000FF0E9EB602D0E82EFCD79E96C69EC95211
:1060C000FF0E9EB602D0E82EFCD725EE33F0050178
:1060D000200E326F9E96C69EC952FF0E9EB602D00B
:1060E000E82EFCD7C9CFDEFF322F6AEF30F0898A65
:1060F0001200899A400EC76E200EC66E9E96C69EEE
:10610000900EC96EFF0E9EB602D0E82EFCD79E966A
:10611000C69E000EC96EFF0E9EB602D0E82EFCD7BA
:106120009E96C69E000EC96EFF0E9EB602D0E82E49
:10613000FCD79E96C69E000EC96EFF0E9EB602D07C
:10614000E82EFCD79E96C69EC952FF0E9EB602D080
:10615000E82EFCD7C9CF2DF59E96C69EC952FF0EDC
:106160009EB602D0E82EFCD7C9CF2EF5898A120040
:10617000ABEC24F0B5C5E8FFD70802E3ABEC24F0A4
:10618000B5C5E8FFC80802E3ABEC24F0B5C5E8FFED
:10619000B90802E3ABEC24F0B5C5E8FFAA0802E3B6
:1061A000ABEC24F0B5C5E8FF9B0802E3ABEC24F0B0
:1061B00023EC29F039EC2DF0F29CF29E8B94C69AD8
:1061C000C290898C9482948C720ED36ED3A4FED725
:1061D00089968A909390FF0EE8CF00F0E82EFED7C4
:1061E000002EFCD78150F294F29A9E909D909E9240
:1061F0009D92F298F292F290F286F28E0300FF00E6
:10BF0000E844F926000C160C2B0C3F0C520C640C68
:10BF1000760C860C960CA50CB30CC10CCF0CDC0C6B
:06BF2000E80CF40C000C1B
:00000001FF
